S01900006F70656E626C745F73746D3332663035312E7372656303
S315080000000020002079050008650500086705000836
S3150800001000000000000000000000000000000000D2
S31508000020000000000000000000000000690500084C
S3150800003000000000000000006B0500086D050008C0
S31508000040C9050008C9050008C9050008C90500084A
S31508000050C9050008C9050008C9050008C90500083A
S31508000060C9050008C9050008C9050008C90500082A
S31508000070C9050008C9050008C9050008C90500081A
S31508000080C9050008C905000800000000C9050008E0
S31508000090C9050008C9050008C9050008C9050008FA
S315080000A0C9050008C9050008C9050008C9050008EA
S315080000B0C905000800000000C90500080000000086
S315080000C010B5064C2378002B07D1054B002B02D020
S315080000D0044800E000BF0123237010BDD0000020B3
S315080000E000000000B01B0008044B10B5002B03D01D
S315080000F00349044800E000BF10BDC04600000000E8
S31508000100D4000020B01B0008002243088B4274D399
S3150800011003098B425FD3030A8B4244D3030B8B42FA
S3150800012028D3030C8B420DD3FF22090212BA030C03
S315080001308B4202D31212090265D0030B8B4219D3E4
S3150800014000E0090AC30B8B4201D3CB03C01A524104
S31508000150830B8B4201D38B03C01A5241430B8B424C
S3150800016001D34B03C01A5241030B8B4201D30B0335
S31508000170C01A5241C30A8B4201D3CB02C01A52415C
S31508000180830A8B4201D38B02C01A5241430A8B421F
S3150800019001D34B02C01A5241030A8B4201D30B0208
S315080001A0C01A5241CDD2C3098B4201D3CB01C01A22
S315080001B0524183098B4201D38B01C01A524143092C
S315080001C08B4201D34B01C01A524103098B4201D31A
S315080001D00B01C01A5241C3088B4201D3CB00C01A87
S315080001E0524183088B4201D38B00C01A52414308FF
S315080001F08B4201D34B00C01A5241411A00D2014624
S31508000200524110467047FFE701B5002000F006F896
S3150800021002BDC0460029F7D076E770477047C0464A
S3150800022010B501F033FA10BD10B501F03DFA10BD56
S3150800023010B59023DB051B69DB0701D5002010BD2F
S3150800024000F03CF80120FAE710B5642000F006F843
S3150800025010BD10B500F008F810BD0000014B18805D
S315080002607047C046EC00002010B501F0C1F90F4BED
S315080002701B68984210D30E4B1B78002B0DD10C4BE4
S3150800028001221A700B4BFF329A6101F0B1F90A4B41
S315080002901B881818054B186010BD054B00221A70EC
S315080002A0044B0132FF329A62EFE7C046F0000020A5
S315080002B0EE00002000080048EC000020024B8022D7
S315080002C052009A627047C04600080048F0B589B0E7
S315080002D01422002103A801F063FC1C4B59698020F5
S315080002E0C003014359615A6902400092009A59694C
S315080002F080208002014359615A6902400192019A9D
S315080003005A69802109030A435A615B690B400293C3
S31508000310029B80277F000E4D00223900280000F03E
S3150800032003FC01260396002404940594902003A94F
S31508000330C00500F033FB039704960594069403A9B9
S31508000340280000F02BFB09B0F0BDC04600100240A3
S3150800035000080048F0B591B01C22002109A801F058
S315080003601FFC1822002103A801F01AFC254BD969A5
S31508000370802292021143D961D969114002910299EA
S315080003805969114359615B691A400192019B04231B
S3150800039003930227049703240594012508959026BC
S315080003A0F60503A9300000F027FC082303930497F9
S315080003B00594002406940794089503A9300000F0D4
S315080003C01BFC96231B0209930A940B940C940C238A
S315080003D00D930E940F940C4C09A9200000F03EFDD5
S315080003E0A3680A4A1340A3606368094A1340636016
S315080003F0A3682A229343A36023682B43236011B082
S31508000400F0BDC0460010024000440040FFFBFFFF5D
S31508000410FFB7FFFF10B5254A136801218B430B432D
S315080004201360224B1B68DB07FBD5214B196880221A
S31508000430D2020A431A601968802252020A431A60D5
S315080004401B4B1B689B03FBD5194B5A68194911406E
S31508000450882252030A435A60DA6A0F218A43DA620B
S315080004601968802252040A431A60114B1B689B01C3
S31508000470FBD50F4B5A68F0218A435A605A680E49D1
S315080004800A405A605A6803218A4301390A435A6066
S31508000490074B5A680C231340082BF9D1074800F07C
S315080004A041FD002000F0A4F810BDC046002002401F
S315080004B000100240FFFFC2FFFFF8FFFF006CDC02DE
S315080004C010B500F0BDF8FFF7A5FFFFF7FFFEFFF731
S315080004D041FFFFF7A5FEFFF7A7FEFCE782B00A4B30
S315080004E0996901221143996199690A400092009A13
S315080004F0DA69802149050A43DA61DB690B40019311
S31508000500019B02B07047C0460010024010B500F0CB
S31508000510C7FB0F4880235B00836200F00BFB90202B
S31508000520C00500F007FB0B4BD9690B480140D961A0
S3150800053059690A4A114059615A6902405A61DA6989
S3150800054007490A40DA619A6901218A439A6110BD0E
S315080005500008004800100240FFFFFDFFFFFFF7FFFD
S31508000560FFFFFFEF7047FEE77047704710B500F0D2
S3150800057077F810BD704700000D4885460D480E49AE
S315080005800E4A002302E0D458C4500433C4188C42DF
S31508000590F9D30B4A0B4C002301E013600432A24244
S315080005A0FBD3FFF7E7FF01F0D7FAFFF789FFFEE76E
S315080005B000200020C0000020D0000020A41D000854
S315080005C0D000002008060020FEE7000010B5074B03
S315080005D001214942196100221A61D960DA609962DB
S315080005E09A62FFF793FF002010BDC0460010024034
S315080005F010B504000F4B1978FA208000FFF784FD28
S3150800060001000D4B1868FFF77FFD00F067F800281A
S315080006100DD1032C01D901200AE001300022210066
S31508000620404200F029F8054B1C60002000E001203C
S3150800063010BDC046C4000020C0000020C80000202D
S3150800064010B5064A136810210B4313600020FFF704
S31508000650CFFFFFF743FF002010BDC0460020024031
S31508000660034A1168034B1B785B1813607047C04632
S31508000670E0050020C400002070B5002811DB8308BF
S31508000680144DC0339B005C5903221040C000FC3255
S3150800069016008640B44389010A40824022435A51D3
S315080006A070BDC0B20F230340083B9B0806339B006E
S315080006B0094A944663445D6803242040C000FF222B
S315080006C014008440A543890111408140294359609B
S315080006D0E6E7C04600E100E000ED00E001380A4B1D
S315080006E098420FD8094A50600948036A1B021B0A38
S315080006F0C02109060B430362002393600733136086
S31508000700002070470120FCE7FFFFFF0010E000E033
S3150800071000ED00E010B5054B0022DA61044A1369C2
S31508000720012423431361018010BDC046E80500205B
S31508000730002002400C4BDB68DB0613D50B4AD36955
S3150800074002210B43D3611023074AD268520706D504
S315080007500649CA6901200243CA6104221343024AB0
S31508000760D36070470023EFE700200240E805002029
S31508000770084B1B691B060BD5064B074A5A60074AE6
S315080007805A601B691B0601D5012002E0002000E023
S31508000790002070470020024023016745AB89EFCD52
S315080007A0034A136980210B43136100207047C04632
S315080007B00020024070B5040000F022FF0500134B2C
S315080007C0DB68DB070AD5631CF9D0002C19D000F0CA
S315080007D017FF401BA042F2D9032011E00B4BDB6840
S315080007E09B0602D5094B2022DA60084BDB68DB063C
S315080007F003D4064BDB685B0705D5FFF79BFF012093
S3150800080070BD0320FCE70020FAE7C046002002403E
S31508000810F0B5C64600B504000D0090461E00214BF3
S315080008201B7E012B3BD01F4B01221A761E48FFF771
S31508000830C1FF00282DD1012C06D0022C02D0042796
S3150800084000241BE00227FBE70127F9E72022D21A3A
S31508000850310091400A004146D940114389B24019F6
S31508000860FFF758FF1048FFF7A5FF104A1369012143
S315080008708B43136100280CD10134E4B2BC4208D280
S3150800088060002301202252429A18DFD43100D14059
S31508000890E4E7044B00221A7604BC9046F0BD022019
S315080008A0FAE7C046E805002050C3000000200240D1
S315080008B0064B0022DA61064B1A6904210A431A61BB
S315080008C01A693C310A431A617047C046E805002098
S315080008D000200240064B0022DA61064B1A69022103
S315080008E00A431A6158611A693E310A431A61704708
S315080008F0E80500200020024070B505000E00244BD4
S315080009001B7E012B41D0224B01221A760368012B4C
S3150800091022D02048FFF74EFF002831D101235B4241
S3150800092033606C680130AB689B026A68944663441E
S31508000930A34226D92000FFF7CDFF1648FFF73AFF56
S31508000940154A136902218B431361002816D18023A7
S31508000950DB009C466444E6E70E48FFF72BFF0028B9
S3150800096001D001200DE0FFF7A3FF0A48FFF722FF99
S31508000970094A136904218B43136102E0346000E0DD
S315080009800120034B00221A7670BD0220FCE7C04600
S31508000990E805002050C3000000200240F0B5CE460E
S315080009A0474680B583B0002333E0032600E00026DF
S315080009B0AE4035003D430234A400554EA551554C72
S315080009C02568D4432E0026404F68FF0301D51543FA
S315080009D02E00504D2E606D682E0026404F68BF03CE
S315080009E001D515432E004B4D6E60AD682E0026408E
S315080009F04F68FF0201D515432E00464DAE60ED68DF
S31508000A002C404E68B60201D52A431400414AD460E8
S31508000A1001330A681400DC4074D001249C4022404B
S31508000A20F6D04D686E1E012E03D9112D01D0122D58
S31508000A3012D185685F000326BE40B5432E00CD68F7
S31508000A40BD40354385604568A5434C6826090124A1
S31508000A5034409C402C434460C7685E000324B4407D
S31508000A60E443A44627408D68B5403D43C5604C68BD
S31508000A70022C01D0122C10D1DC080834A400A1469F
S31508000A80275807251D40AD000F24AC40A7430C6925
S31508000A90AC4025003D434C46255005686446254034
S31508000AA003244F683C40B4402C4304604C68E4007F
S31508000AB0AED5194DAE6901242643AE61AD692C4009
S31508000AC00194019C9C08A51CAD00114EAF59032545
S31508000AD01D40AD000F26AE40B7439026F605B0423E
S31508000AE000D164E70D4EB04208D00D4EB04207D093
S31508000AF00C4EB04200D158E7052659E7012657E7BC
S31508000B00022655E703B00CBC90469946F0BDC04690
S31508000B1000000140000401400010024000040048A3
S31508000B2000080048000C0048002A01D1816270477D
S31508000B308161FCE79023DB0598420DD0244B98424F
S31508000B4016D0244B98421FD0234B984228D0234BCB
S31508000B50984231D001200AE0214B996A80229202FC
S31508000B600A439A629A6A1F490A409A6200207047A5
S31508000B701B4B996A8022D2020A439A629A6A1A49D8
S31508000B800A409A620020F2E7154B996A80221203FE
S31508000B900A439A629A6A15490A409A620020E6E769
S31508000BA00F4B996A802252030A439A629A6A10493D
S31508000BB00A409A620020DAE7094B996A8022D20332
S31508000BC00A439A629A6A0B490A409A620020CEE75B
S31508000BD00004004800080048000C004800140048BB
S31508000BE000100240FFFFFDFFFFFFFBFFFFFFF7FFBF
S31508000BF0FFFFEFFFFFFFBFFFF0B5002214E0C66856
S31508000C001C005C4365002D19ED432E400F696743B0
S31508000C103E43C6604E68022E24D003681D404B68CA
S31508000C205C432C43046001320B681C00D44035D069
S31508000C30012494402340F6D04C68013C012CDED8B0
S31508000C4084681D005D436E007619B4438E6875434B
S31508000C502C4384600D684468AC43CE6875432C43C6
S31508000C604460CCE7FF2B0BD8076A26005E43734324
S31508000C701E01F61AB7434E6973433B430362CCE73A
S31508000C80476A1B0A1E005E435E4373431E01F61A3B
S31508000C90B7434E6973433B434362BEE70020F0BD4A
S31508000CA082B0284A136801210B431360254B1B6841
S31508000CB09B07FBD5234A1368F8218B4378390B43E6
S31508000CC0136001235B420193019B1F490B4001936B
S31508000CD0019B53601B4B5B680C221A42FAD1194AD6
S31508000CE013680193019B19490B400193019B1360FB
S31508000CF0144B1B689B01FBD4124B1A6814490A4013
S31508000D001A60002159605A6BF820824378380243EA
S31508000D105A635A6B7F3882435A635A6B033082434D
S31508000D205A63D9621963BF2212040192019A9A6022
S31508000D309960596A802252040A435A62002002B016
S31508000D407047C046001002400CF8FFF0FFFFF6FEA1
S31508000D50FFFFFBFF044B5A6812090F231340034A8F
S31508000D60D35CD8407047C04600100240C81B000834
S31508000D70044B5A68120A07231340034AD35CD84027
S31508000D807047C04600100240D81B000870B50B4BD0
S31508000D905B68802252021340934201D0084800E063
S31508000DA00848064DE96A0F2421400131FFF7ACF9DE
S31508000DB06B689B0C1C400234604370BD00100240F7
S31508000DC000093D0000127A0010B5054B5A680C233D
S31508000DD01340082B02D1FFF7D9FF10BD0148FCE7E5
S31508000DE00010024000127A0010B50400FFF7ECFF6D
S31508000DF02060FFF7AFFF6060FFF7BAFFA06010BD85
S31508000E0010B5002823D1134B1A6B032383401340D4
S31508000E1002061343022B13D0032B0BD0012B06D04B
S31508000E20FFF7D2FFFFF796FFFFF7A2FF10E0FFF7E5
S31508000E30CBFF0DE0074B1B689B0709D5064807E063
S31508000E40044B1B6A9B0703D58020000200E00020A4
S31508000E5010BDC0460010024000127A0030B585B0B9
S31508000E6004000D000368DB0748D40368274A1A40C4
S31508000E704B68C9680B4329690B43A9690B4313439C
S31508000E8003604368224A1340AA6813434360836891
S31508000E90204A13406A69134383601F4B984204D063
S31508000EA01E4B984217D0012029E00020FFF7A8FF23
S31508000EB0002826D02968002925D0AA6980231B0284
S31508000EC09A420DD04B08C018FFF71EF90004000C13
S31508000ED0E060002013E001A8FFF786FF0398E7E724
S31508000EE040004B08C018FFF70FF90D4B03404008A8
S31508000EF0072210401843E060002000E0012005B0FA
S31508000F0030BD0120FBE70120F9E7C046F369FFFF82
S31508000F10FFCFFFFFFFFCFFFF003801400044004001
S31508000F20F0FF0000014B18607047C046C000002063
S31508000F3072B6704762B6704710B5FFF7F9FF10BD75
S31508000F4070B508E04D1C461C0B78037000F00DFCCC
S31508000F50300029002200541EA4B2002AF2D170BD26
S31508000F6010B582B000F052FA002801D102B010BDC7
S31508000F70FFF75EF90028F9D000F0C4FBFFF726FB5F
S31508000F8000F00CFB0E4A916901231943916192699D
S31508000F9013400193019B00F03DFA01008020C02216
S31508000FA08005FFF7CDFF074A136803218B430B43E0
S31508000FB0136000F02FFA4468FFF7BCFFA047D5E797
S31508000FC0001002400000014070B50500002401E051
S31508000FD00134E4B20C2C15D800F0C7FB63001B19CA
S31508000FE09A00094BD358AB42F2D862001219900006
S31508000FF0054A121852689B18AB42E9D9024B1B18CE
S31508001000187A00E0FF2070BDE01B000870B50500E7
S3150800101000240C2C10D800F0A8FB63001B199A00BA
S31508001020074B9B181B7AAB4202D00134E4B2F0E7B7
S315080010301300034A985801E00120404270BDC0469B
S31508001040E01B000870B5050000240C2C10D800F031
S315080010508CFB63001B199A00064B9B181B7AAB4244
S3150800106002D00134E4B2F0E7024B9B18586800E05E
S31508001070002070BDE01B000810B5CB0509D1036838
S315080010808B4208D002C080229200FFF759FF012048
S3150800109000E0002010BD0120FCE7F8B50700006855
S315080010A0FFF792FFFF2821D0FFF762FB00257F2D6F
S315080010B013D8AB003A68D418FB185E6800F055FBE5
S315080010C03200002321000220FFF7A2FB002806D1E8
S315080010D02368B34208D10135E9E7012400E000247A
S315080010E0FFF75EFB2000F8BD0024F9E70024F9E7C6
S315080010F070B504000D000C4B984211D00B4B994269
S3150800110008D1094C29002000FFF7B6FF002809D0AE
S31508001110200070BDFFF7C1FF0028F3D10024F7E7D0
S31508001120034CEFE70024F3E7F8020020002000084C
S31508001130F4000020F0B5C64600B507000C001500FF
S315080011401E004B0A5B0298460368013307D03B68CA
S3150800115043450AD13B68E41A3C19043414E0414675
S31508001160FFF78AFF0028F2D120E041463800FFF752
S31508001170BFFF071EEED1002018E02B78237001343C
S315080011800135013E002E10D000F0EFFA3B1DE31AA0
S31508001190094A9342F1D98021890041443800FFF772
S315080011A0A7FF071E05D0041DE7E7012004BC9046EB
S315080011B0F0BD0020FAE7C046FF010000F0B587B091
S315080011C00D0000230593884232D80124032835D917
S315080011D0102D37D8012C32D1FFF718FF0700280049
S315080011E0FFF714FF06002800FFF72CFF3618013E0C
S315080011F0F61B0136B60AB6B20023029303970133EB
S315080012000493FFF7B5FA0025B54214D200F0ADFAFB
S3150800121005A902A8FFF770FB00280BD1039B0193D1
S315080012208022D2009446634403930135ADB2EBE7BE
S315080012300024CBE70024FFF7B3FA00E000242000DF
S3150800124007B0F0BD0024FAE701235B42024A1360A7
S31508001250024A13607047C046F4000020F8020020D6
S3150800126070B504000E0015004A1E134B1B1A9A424D
S3150800127001D9002070BDFFF7A7FEFF2818D0301946
S315080012800138FFF7A1FEFF2814D0630A5B020B4A58
S31508001290934206D033002A0021000948FFF74AFF87
S315080012A0E8E733002A0021000648FFF743FFE1E795
S315080012B00020DFE70020DDE7FFFF00080020000828
S315080012C0F4000020F8020020F8B506000C004A1EBB
S315080012D00C4B1B1A9A4201D90020F8BDFFF774FE81
S315080012E00500A0190138FFF76FFEFF2D06D0FF286D
S315080012F006D001002800FFF761FFEEE70020ECE7C3
S315080013000020EAE7FFFF000800B583B0104B1B6812
S3150800131001331BD00E4A536891688C466344D168E2
S315080013208C46634411698C46634451698C46634410
S3150800133091698C466344D2699B185B42019301AA62
S3150800134004210448FFF78CFF03B000BD0120FBE72A
S31508001350F8020020C02000080E4B1A680E4B1B68C6
S31508001360D2180E4B1B689A180D4B1B689B180D4A12
S315080013701268D3180C4A1268D2180C4B1B689A18B4
S315080013800B4B1B689B18002B01D0002070470120CF
S31508001390FCE7C046002000080420000808200008D2
S315080013A00C20000810200008142000081820000847
S315080013B0C020000810B50B4B1B6801330AD10A4B35
S315080013C01B6801330CD00848FFF767FE002808D0D1
S315080013D0012006E00348FFF760FE0028EFD100E091
S315080013E0012010BDF8020020F400002000487047D4
S315080013F00020000810B5FFF727FF10BD10B5FFF74E
S315080014002FFF10BD10B5FFF75FFF10BD10B5FFF732
S31508001410A3FF10BD10B5FFF7E9FF10BD10B5FFF724
S3150800142073FF002800D110BDFFF7C4FFFBE70000DB
S31508001430054BDB699B0604D5034B9B8C0370012087
S3150800144070470020FCE7C0460044004010B580B253
S31508001450084B188500F0CCF80A300400054BDB6908
S315080014601B0605D400F081F900F0C2F8A042F5D9B0
S3150800147010BDC0460044004030B589B00C4C236806
S315080014800125AB432360E1231B020193002302934A
S31508001490039304930C2205920693079301A920004F
S315080014A0FFF7DCFC23682B43236009B030BDC04638
S315080014B00044004070B506000D00402904D82800F5
S315080014C0FFF7C4FF00240BE08421074800F09CF8CE
S315080014D0F5E700F04AF9305DFFF7B8FF0134A4B22A
S315080014E0ABB2A342F5D870BD7C1C000870B50600E7
S315080014F00D00264B1C78002C17D12548FFF798FFBE
S31508001500012801D0200070BD214B1B78013BDBB2BE
S315080015103F2BF7D800F06CF81E4B18601E4B0022C4
S315080015201A701A4B01321A70ECE71B4B1B78013301
S315080015301748C018FFF77CFF0400012817D1164B7F
S315080015401A780132D2B21A70114B1B789A4201D01E
S315080015500024D7E792B20E4901313000FFF7F0FCBC
S315080015600A4B00221A700C4B1B782B70CAE700F046
S315080015703FF8084B1B686433984204D9034B002292
S315080015801A700024BEE70024BCE7C0463D050020CB
S31508001590FC040020400500203E050020024B0022E6
S315080015A01A605A609A60704710E000E010B5FFF7BD
S315080015B0F5FF054B054A5A6000229A600521196015
S315080015C0034B1A6010BDC04610E000E07FBB000068
S315080015D044050020044B1B68DB0303D5034A136844
S315080015E0013313607047C04610E000E04405002050
S315080015F010B5FFF7EFFF014B186810BD4405002032
S3150800160010B5FFF7F5FF10BD10B500F0AEF8FCE712
S3150800161010B500F09FF8012803D00B4B1B78012B5F
S3150800162000D010BDFFF7E4FF084B1B68084A126894
S315080016309B18F533FF339842F3D3034B00221A70F5
S31508001640FFF78EFCEDE7C0464C0500204805002054
S315080016505005002010B5054B1B78012B00D010BD96
S31508001660FFF7C6FF024B1860F9E7C0464C05002095
S315080016705005002010B5044B01221A70FFF7EAFF47
S31508001680FFF7C6FF10BDC0464C05002010B5FFF792
S3150800169053FC00F066F8FFF789FFFFF7ABFE00F092
S315080016A00DF8FFF7E7FF10BD10B500F05EF8FFF77D
S315080016B091FF00F00FF8FFF7ABFF10BD10B500F073
S315080016C0CFF9FFF7D9FE024B00221A7010BDC046AB
S315080016D0CC00002000B583B06B46D91D0748FFF73C
S315080016E005FF012801D003B000BD054B00221A7082
S315080016F06B46D979014800F0D3F9F4E75405002080
S31508001700CC0000207047000010B5054B1B78002B55
S3150800171002D000F0BDF910BDC9B2FFF7CBFEF8E75D
S31508001720CC000020044B1B78013BDBB2022B01D90D
S31508001730402000E000207047CC000020044B1B78B6
S31508001740013BDBB2022B01D9402000E000207047A4
S31508001750CC00002010B500F091F9002800D0012037
S3150800176010BD10B5FEF770FD10BD10B5FEF771FD82
S3150800177010BD0000014B00225A70704794050020E6
S31508001780034BFE22DA701871BA3A02219952704751
S315080017909405002010B5054C00232370FFF7EAFFD7
S315080017A0FF23E370BB3B0122E25210BD94050020E3
S315080017B0064BFF22DA7000221A71597859719A710C
S315080017C0DA711A724432062199527047940500203C
S315080017D010B50020FFF7D4FF10BD0000094BFF220B
S315080017E0DA70094A9A6400221A715A719A710721A5
S315080017F0D971002119725972997244220831995285
S315080018007047C04694050020941D0008044BFF222B
S31508001810DA7042689A644422012199527047C04698
S315080018209405002010B53120FFF7AAFF10BD00006F
S3150800183070B5084CFF23E370002525716571FFF725
S3150800184071FFA071E5712572657244230722E25281
S3150800185070BDC0469405002070B5FFF78BFF0D4C90
S3150800186001252570FF23E370EF3B23710023637185
S31508001870FFF758FFA071FFF761FFE071FFF75EFF02
S31508001880000A20726572A57244230822E252FFF705
S31508001890B1FD70BD9405002070B505004478FFF7CA
S315080018A041FF0138844211DC6A780A4C201DA16C7C
S315080018B0FFF746FBFF23E3706B78A26C94466344FC
S315080018C0A3646B7801334422A35270BD2220FFF72C
S315080018D057FFFAE79405002070B504004578FFF72E
S315080018E021FF0138854212DC61680B4DA9646278D4
S315080018F0281DFFF725FBFF23EB706378AA6C944637
S315080019006344AB64637801334422AB5270BD222032
S31508001910FFF736FFFAE7C04694050020F8B505003C
S315080019201700002406E02B781C19E4B20135FFF7EE
S315080019301CFF31004E1E0029F5D13C600120F8BD80
S3150800194010B5084CFF23E370E21D4168A06CFFF751
S31508001950E5FF207100236371A37144330822E25224
S3150800196010BDC0469405002070B504000E4B9D6C52
S31508001970FFF7D8FE411E621C2800FFF73FFD00282E
S315080019800DD0094CFF23E370FFF7CCFE0138A36C9A
S315080019909C466044A06444230122E25270BD313063
S315080019A0FFF7EEFEFAE7C0469405002070B504007E
S315080019B04578FFF7B7FE0238854210DC134BFF2245
S315080019C0DA70BB3A01219952617800290BD1FFF7E9
S315080019D025FD002806D13130FFF7D2FE02E022208D
S315080019E0FFF7CEFE70BD094B986CA21CFFF706FDEB
S315080019F0002806D06378054A916C8C466344936444
S31508001A00F0E73130FFF7BCFEECE7C046940500204E
S31508001A1010B5094B9B6C41681800FFF7F3FC0028CA
S31508001A2006D0054BFF22DA70BB3A0121995210BD48
S31508001A303130FFF7A5FEFAE79405002010B5FFF749
S31508001A408FFA034BFF22DA70BB3A0121995210BD77
S31508001A509405002010B589B2FFF756FE10BD0000A8
S31508001A60054B00221A709A6443215A5401315A527E
S31508001A709A705A707047C04694050020034B1B782D
S31508001A80002B01D0012070470020FCE794050020B8
S31508001A90024A43230021D1547047C04694050020CA
S31508001AA010B50378FF2B04D0294A1278012A14D0DE
S31508001AB010BDFFF7D1FE264A4323D35C012B42D043
S31508001AC0234A4423D15E0029F2DD10004323012274
S31508001AD0C2540330FFF7BEFFEAE73733DAB2352AD6
S31508001AE02DD893001B4AD3589F46FFF7D5FEE2E749
S31508001AF0FFF7F2FEDFE7FFF789FEDCE7FFF720FFD7
S31508001B00D9E7FFF76BFED6E7FFF762FED3E7FFF7E5
S31508001B104FFED0E7FFF73EFECDE7FFF725FFCAE702
S31508001B20FFF744FFC7E7FFF783FEC4E7FFF770FF39
S31508001B30C1E7FFF783FFBEE7FFF774FEBBE7202088
S31508001B40FFF71EFEB7E71020FFF71AFEB8E7C046F4
S31508001B5094050020BC1C000870B500260C4D0D4CE1
S31508001B60641BA410A64209D1002600F021F80A4DEC
S31508001B700A4C641BA410A64205D170BDB300EB58ED
S31508001B8098470136EEE7B300EB5898470136F2E777
S31508001B909C1D00089C1D00089C1D0008A01D00082F
S31508001BA003001218934200D1704719700133F9E700
S31508001BB0F8B5C046F8BC08BC9E467047F8B5C0469E
S30D08001BC0F8BC08BC9E467047FC
S31508001BC800000000000000000102030406070809D7
S31508001BD800000000010203040020000800080000B5
S31508001BE8040000000028000800080000050000009E
S31508001BF80030000800080000060000000038000849
S31508001C08000800000700000000400008000800005F
S31508001C180800000000480008000800000900000045
S31508001C2800500008000800000A00000000580008D4
S31508001C38000800000B00000000600008000800000B
S31508001C480C00000000680008000800000D000000ED
S31508001C5800700008000800000E0000000078000860
S31508001C68000800000F00000000800008008000003F
S31508001C7810000000433A2F576F726B2F736F667404
S31508001C88776172652F4F70656E424C542F54617296
S31508001C986765742F536F757263652F41524D434DAF
S31508001CA8305F53544D333246302F72733233322EE7
S31508001CB8630000001A1B00083E1B00083E1B0008AC
S31508001CC8381B00083E1B00083E1B0008321B00088C
S31508001CD8201B00082C1B0008261B00083E1B0008B2
S31508001CE83E1B00083E1B00083E1B00083E1B00085A
S31508001CF83E1B00083E1B00083E1B00083E1B00084A
S31508001D083E1B00083E1B00083E1B00083E1B000839
S31508001D183E1B00083E1B00083E1B00083E1B000829
S31508001D283E1B00083E1B00083E1B00083E1B000819
S31508001D383E1B00083E1B00083E1B00083E1B000809
S31508001D483E1B00083E1B00083E1B00083E1B0008F9
S31508001D583E1B00083E1B00083E1B0008FC1A00082C
S31508001D68F01A0008EA1A0008F61A00083E1B0008C6
S31508001D783E1B00083E1B0008021B00083E1B000805
S31508001D88081B00080E1B0008141B00084F70656E18
S30908001D98424C540057
S30908001D9CE900000844
S30908001DA0C100000868
S31508001DA400127A000100000004000000040000008C
S7050800057974
